C51 COMPILER V9.51   PIN_1                                                                 12/22/2013 21:56:17 PAGE 1   


C51 COMPILER V9.51, COMPILATION OF MODULE PIN_1
OBJECT MODULE PLACED IN .\DP8051\DP8051_Keil_951\Debug\Pin_1.obj
COMPILER INVOKED BY: C:\Program Files (x86)\Cypress\PSoC Creator\3.0\PSoC Creator\import\keil\pk51\9.51\C51\BIN\c51.exe 
                    -.\Generated_Source\PSoC3\Pin_1.c NOIV LARGE MODDP2 OMF2 VB(1) PR(.\DP8051\DP8051_Keil_951\Debug\Pin_1.lst) CD DB NOIP OT
                    -(2,SIZE) DF(DEBUG) INCDIR(.,.\Generated_Source\PSoC3) OJ(.\DP8051\DP8051_Keil_951\Debug\Pin_1.obj)

line level    source

   1          /*******************************************************************************
   2          * File Name: Pin_1.c  
   3          * Version 1.90
   4          *
   5          * Description:
   6          *  This file contains API to enable firmware control of a Pins component.
   7          *
   8          * Note:
   9          *
  10          ********************************************************************************
  11          * Copyright 2008-2012, Cypress Semiconductor Corporation.  All rights reserved.
  12          * You may use this file only in accordance with the license, terms, conditions, 
  13          * disclaimers, and limitations in the end user license agreement accompanying 
  14          * the software package with which this file was provided.
  15          *******************************************************************************/
  16          
  17          #include "cytypes.h"
  18          #include "Pin_1.h"
  19          
  20          
  21          /*******************************************************************************
  22          * Function Name: Pin_1_Write
  23          ********************************************************************************
  24          *
  25          * Summary:
  26          *  Assign a new value to the digital port's data output register.  
  27          *
  28          * Parameters:  
  29          *  prtValue:  The value to be assigned to the Digital Port. 
  30          *
  31          * Return: 
  32          *  None 
  33          *  
  34          *******************************************************************************/
  35          void Pin_1_Write(uint8 value) 
  36          {
  37   1          uint8 staticBits = (Pin_1_DR & (uint8)(~Pin_1_MASK));
  38   1          Pin_1_DR = staticBits | ((uint8)(value << Pin_1_SHIFT) & Pin_1_MASK);
  39   1      }
  40          
  41          
  42          /*******************************************************************************
  43          * Function Name: Pin_1_SetDriveMode
  44          ********************************************************************************
  45          *
  46          * Summary:
  47          *  Change the drive mode on the pins of the port.
  48          * 
  49          * Parameters:  
  50          *  mode:  Change the pins to this drive mode.
  51          *
  52          * Return: 
  53          *  None
C51 COMPILER V9.51   PIN_1                                                                 12/22/2013 21:56:17 PAGE 2   

  54          *
  55          *******************************************************************************/
  56          void Pin_1_SetDriveMode(uint8 mode) 
  57          {
  58   1              CyPins_SetPinDriveMode(Pin_1_0, mode);
  59   1              CyPins_SetPinDriveMode(Pin_1_1, mode);
  60   1      }
  61          
  62          
  63          /*******************************************************************************
  64          * Function Name: Pin_1_Read
  65          ********************************************************************************
  66          *
  67          * Summary:
  68          *  Read the current value on the pins of the Digital Port in right justified 
  69          *  form.
  70          *
  71          * Parameters:  
  72          *  None 
  73          *
  74          * Return: 
  75          *  Returns the current value of the Digital Port as a right justified number
  76          *  
  77          * Note:
  78          *  Macro Pin_1_ReadPS calls this function. 
  79          *  
  80          *******************************************************************************/
  81          uint8 Pin_1_Read(void) 
  82          {
  83   1          return (Pin_1_PS & Pin_1_MASK) >> Pin_1_SHIFT;
  84   1      }
  85          
  86          
  87          /*******************************************************************************
  88          * Function Name: Pin_1_ReadDataReg
  89          ********************************************************************************
  90          *
  91          * Summary:
  92          *  Read the current value assigned to a Digital Port's data output register
  93          *
  94          * Parameters:  
  95          *  None 
  96          *
  97          * Return: 
  98          *  Returns the current value assigned to the Digital Port's data output register
  99          *  
 100          *******************************************************************************/
 101          uint8 Pin_1_ReadDataReg(void) 
 102          {
 103   1          return (Pin_1_DR & Pin_1_MASK) >> Pin_1_SHIFT;
 104   1      }
 105          
 106          
 107          /* If Interrupts Are Enabled for this Pins component */ 
 108          #if defined(Pin_1_INTSTAT) 
              
                  /*******************************************************************************
                  * Function Name: Pin_1_ClearInterrupt
                  ********************************************************************************
                  *
                  * Summary:
                  *  Clears any active interrupts attached to port and returns the value of the 
C51 COMPILER V9.51   PIN_1                                                                 12/22/2013 21:56:17 PAGE 3   

                  *  interrupt status register.
                  *
                  * Parameters:  
                  *  None 
                  *
                  * Return: 
                  *  Returns the value of the interrupt status register
                  *  
                  *******************************************************************************/
                  uint8 Pin_1_ClearInterrupt(void) 
                  {
                      return (Pin_1_INTSTAT & Pin_1_MASK) >> Pin_1_SHIFT;
                  }
              
              #endif /* If Interrupts Are Enabled for this Pins component */ 
 131          
 132          
 133          /* [] END OF FILE */
C51 COMPILER V9.51   PIN_1                                                                 12/22/2013 21:56:17 PAGE 4   

ASSEMBLY LISTING OF GENERATED OBJECT CODE


             ; FUNCTION _Pin_1_Write (BEGIN)
                                           ; SOURCE LINE # 35
0000 900000      R     MOV     DPTR,#value
0003 EF                MOV     A,R7
0004 F0                MOVX    @DPTR,A
                                           ; SOURCE LINE # 36
                                           ; SOURCE LINE # 37
0005 9051C0            MOV     DPTR,#051C0H
0008 E0                MOVX    A,@DPTR
0009 FF                MOV     R7,A
000A EF                MOV     A,R7
000B 54F3              ANL     A,#0F3H
000D FF                MOV     R7,A
000E 900000      R     MOV     DPTR,#staticBits
0011 EF                MOV     A,R7
0012 F0                MOVX    @DPTR,A
                                           ; SOURCE LINE # 38
0013 900000      R     MOV     DPTR,#value
0016 E0                MOVX    A,@DPTR
0017 FF                MOV     R7,A
0018 EF                MOV     A,R7
0019 25E0              ADD     A,ACC
001B 25E0              ADD     A,ACC
001D FF                MOV     R7,A
001E EF                MOV     A,R7
001F 540C              ANL     A,#0CH
0021 FF                MOV     R7,A
0022 900000      R     MOV     DPTR,#staticBits
0025 E0                MOVX    A,@DPTR
0026 FE                MOV     R6,A
0027 EF                MOV     A,R7
0028 4E                ORL     A,R6
0029 FF                MOV     R7,A
002A 9051C0            MOV     DPTR,#051C0H
002D EF                MOV     A,R7
002E F0                MOVX    @DPTR,A
                                           ; SOURCE LINE # 39
002F 22                RET     
             ; FUNCTION _Pin_1_Write (END)

             ; FUNCTION _Pin_1_SetDriveMode (BEGIN)
                                           ; SOURCE LINE # 56
0000 900000      R     MOV     DPTR,#mode
0003 EF                MOV     A,R7
0004 F0                MOVX    @DPTR,A
                                           ; SOURCE LINE # 57
                                           ; SOURCE LINE # 58
0005 900000      R     MOV     DPTR,#mode
0008 E0                MOVX    A,@DPTR
0009 FF                MOV     R7,A
000A EF                MOV     A,R7
000B 540E              ANL     A,#0EH
000D FF                MOV     R7,A
000E 905062            MOV     DPTR,#05062H
0011 E0                MOVX    A,@DPTR
0012 FE                MOV     R6,A
0013 EE                MOV     A,R6
0014 54F1              ANL     A,#0F1H
0016 FE                MOV     R6,A
C51 COMPILER V9.51   PIN_1                                                                 12/22/2013 21:56:17 PAGE 5   

0017 EE                MOV     A,R6
0018 4F                ORL     A,R7
0019 FF                MOV     R7,A
001A 905062            MOV     DPTR,#05062H
001D EF                MOV     A,R7
001E F0                MOVX    @DPTR,A
                                           ; SOURCE LINE # 59
001F 900000      R     MOV     DPTR,#mode
0022 E0                MOVX    A,@DPTR
0023 FF                MOV     R7,A
0024 EF                MOV     A,R7
0025 540E              ANL     A,#0EH
0027 FF                MOV     R7,A
0028 905063            MOV     DPTR,#05063H
002B E0                MOVX    A,@DPTR
002C FE                MOV     R6,A
002D EE                MOV     A,R6
002E 54F1              ANL     A,#0F1H
0030 FE                MOV     R6,A
0031 EE                MOV     A,R6
0032 4F                ORL     A,R7
0033 FF                MOV     R7,A
0034 905063            MOV     DPTR,#05063H
0037 EF                MOV     A,R7
0038 F0                MOVX    @DPTR,A
                                           ; SOURCE LINE # 60
0039 22                RET     
             ; FUNCTION _Pin_1_SetDriveMode (END)

             ; FUNCTION Pin_1_Read (BEGIN)
                                           ; SOURCE LINE # 81
                                           ; SOURCE LINE # 82
                                           ; SOURCE LINE # 83
0000 9051C1            MOV     DPTR,#051C1H
0003 E0                MOVX    A,@DPTR
0004 FF                MOV     R7,A
0005 EF                MOV     A,R7
0006 540C              ANL     A,#0CH
0008 FF                MOV     R7,A
0009 7E00              MOV     R6,#00H
000B EF                MOV     A,R7
000C 7802              MOV     R0,#02H
000E         ?C0005:
000E CE                XCH     A,R6
000F C3                CLR     C
0010 13                RRC     A
0011 CE                XCH     A,R6
0012 13                RRC     A
0013 D8F9              DJNZ    R0,?C0005
0015 FF                MOV     R7,A
                                           ; SOURCE LINE # 84
0016         ?C0003:
0016 22                RET     
             ; FUNCTION Pin_1_Read (END)

             ; FUNCTION Pin_1_ReadDataReg (BEGIN)
                                           ; SOURCE LINE # 101
                                           ; SOURCE LINE # 102
                                           ; SOURCE LINE # 103
0000 9051C0            MOV     DPTR,#051C0H
0003 E0                MOVX    A,@DPTR
0004 FF                MOV     R7,A
C51 COMPILER V9.51   PIN_1                                                                 12/22/2013 21:56:17 PAGE 6   

0005 EF                MOV     A,R7
0006 540C              ANL     A,#0CH
0008 FF                MOV     R7,A
0009 7E00              MOV     R6,#00H
000B EF                MOV     A,R7
000C 7802              MOV     R0,#02H
000E         ?C0006:
000E CE                XCH     A,R6
000F C3                CLR     C
0010 13                RRC     A
0011 CE                XCH     A,R6
0012 13                RRC     A
0013 D8F9              DJNZ    R0,?C0006
0015 FF                MOV     R7,A
                                           ; SOURCE LINE # 104
0016         ?C0004:
0016 22                RET     
             ; FUNCTION Pin_1_ReadDataReg (END)



MODULE INFORMATION:   STATIC OVERLAYABLE
   CODE SIZE        =    152    ----
   CONSTANT SIZE    =   ----    ----
   XDATA SIZE       =   ----       3
   PDATA SIZE       =   ----    ----
   DATA SIZE        =   ----    ----
   IDATA SIZE       =   ----    ----
   BIT SIZE         =   ----    ----
   EDATA SIZE       =   ----    ----
   HDATA SIZE       =   ----    ----
   XDATA CONST SIZE =   ----    ----
   FAR CONST SIZE   =   ----    ----
END OF MODULE INFORMATION.


C51 COMPILATION COMPLETE.  0 WARNING(S),  0 ERROR(S)
